:10000000830100308A000428203084003730162015
:1000100083010730C900EF30C80037308400483012
:100020001A208301FF2B04068001840A04060319A9
:1000300000341328F00024208000840A040870068D
:10004000031900341B28C800C91B2F28491B372857
:1000500049088A004808C80A0319C90A820083139C
:10006000491883174808C80A840000080800253486
:1000700064344C346934723461342034253464344B
:100080004B34753472347534733400344434693409
:100090006A346934743461346C3420344B347534CC
:0C00A0006D346234613472346134003419
:1005BC008312080083120313A9000511803E302B0F
:1005CC00831203130511013030230230F92AF00095
:1005DC000030711870070310F00D0310F10CF108C6
:1005EC0003190800EF2A83120313A9000430AA0090
:1005FC005330AB00AB0B002BAA0BFE2AA90BFC2A29
:10060C000800831203130515132B2A08C9002908A7
:10061C00A90A0319AA0A232030232A08C900290889
:10062C0023200038031908000B2BF401F5010310EB
:10063C00F30CF20C031C292B7008F4077108031837
:10064C00710AF5070310F00DF10D7208730403190C
:10065C0000341D2B83120313AB002B0E0F39F0004B
:10066C000608F03970048600851585112B080F39A2
:10067C00F0000608F03970048600851585110D30E0
:10068C00AC00AC0B472B080083120313A500051517
:10069C00250E0F39F0000608F03970048600851518
:1006AC00851125080F39F0000608F0397004860012
:1006BC00851585110D30A600A60B622B0800831240
:1006CC00031305110F30F9220330860085158511AF
:1006DC000530F922851585112130A500A50B742B49
:1006EC00851585110530F922023086008515851196
:1006FC000D30A500A50B802B28303023083030237B
:10070C000F3030230630302BE622F301C830F400D2
:10071C004230F5002208F0002308F1002408F20012
:10072C0003273B277008A1006430F200F301210875
:10073C00F000F1011B237408F0007508F100A226EB
:10074C007008F3007108F4007208F5002208F0003C
:10075C002308F1002408F200D6263B277008A000DD
:10076C000030E0224630A9000030AA0007233730C1
:10077C00AA000030AB002008A700A8012108A500A2
:10078C00A6012530A9003730D0244030E022373084
:10079C00A9008030AA00072383169C18D32B0130A4
:1007AC009B008312210883169A0003108B1B0314E1
:1007BC008B131C1555309D00AA309D009C141C11E8
:1007CC0003188B179C18E82B02309B00831220080F
:1007DC0083169A0003108B1B03148B131C155530B6
:1007EC009D00AA309D009C141C1103188B178312BA
:0407FC0008001330AE
:10080000831603138500F0308600073083129F00A3
:1008100085018601FA30F9226523E622051A352C76
:1008200083169C18112C01309B009A0103108B1B1E
:1008300003148B131C1555309D00AA309D009C1489
:100840001C1103188B179C18232C02309B009A0153
:1008500003108B1B03148B131C1555309D00AA30FD
:100860009D009C141C1103188B1783169B011C14EC
:100870001A08593A031D612C01309B001C141A08F8
:100880008312A100023083169B001C141A088312E5
:10089000A0006430F200F3012108F000F1011B23F5
:1008A0002008F000F1017408F0070318F10A750838
:1008B000F107A2267008A2007108A3007208A40024
:1008C000782C9C18612C9B0159309A0003108B1BCB
:1008D00003148B131C1555309D00AA309D009C14E9
:1008E0001C1103188B1700308312A201A301A4016D
:1008F0008A23051C872C05187B2CF3018030F4001B
:100900003F30F500223084008313FA268A23851CA9
:10091000952C8518892CF301A030F4004030F500A7
:10092000223084008313FA268A23061EA32C061A7B
:10093000972CF3012030F4004130F5002230840080
:100940008313FA268A23861EB12C861AA52CF3015E
:10095000C830F4004130F500223084008313FA26B9
:100960008A23061FBF2C061BB32CF3014830F4006A
:100970004230F500223084008313FA268A23861F32
:10098000CD2C861BC12CF301C830F4004230F50099
:10099000223084008313FA268A236430F922792CCA
:1009A0008312B200B00103132908AD00812E310873
:1009B000253A031D742EFF30AE00AF01AC013E2E70
:1009C000B2080319E72C3208840083138001300831
:1009D00008000230AD072D02840083130008722E38
:1009E000AC0AF62C0830AE07FE30AE070230AD0779
:1009F0002D02840083130008B300840A0008B400A9
:100A00002C18B41F0A2DB309B409B30A0319B40A88
:100A1000AF030B2DAC010B30AE072E08F200F30133
:100A20003408F1003308F000AA277008B1002E083E
:100A3000F200F3013308F0003408F100AA2774082B
:100A4000B3007508B400B501B50AB6013608340222
:100A5000031D2C2D35083302031C492D2E08F200EE
:100A6000F3013508F0003608F1001B237408B500C7
:100A70007508B600AF03262DB00AB2080319472D3A
:100A800032088400831320308000B20A492D2030C0
:100A9000DE22AF032F08803A7F3E03183C2D2C1C2A
:100AA0005E2DB00AB20803195C2D3208840083134E
:100AB0002D308000B20A5E2D2D30DE222E08F2008D
:100AC000F3013508F0003608F100AA277408B500D4
:100AD0007508B60035040319932D3608F300350860
:100AE000F2003408F1003308F000AA277408F0007F
:100AF0007508F1002E08F200F301AA277008AF0074
:100B0000803A763E031C862D0730AF07B00AB20844
:100B10000319902D3208840083132F08303E592D7D
:100B20002F08303E5D2D0A303102031C992D07300D
:100B3000B107B00AB2080319A32D32088400831349
:100B40003108303E7C2E3108303E802EB00AB2088B
:100B50000319B12D32088400831320308000B20ABB
:100B6000B32D2030DE22AF032F08803A7E3E0318DB
:100B7000A62D0230AD072D02840083130008B100BA
:100B8000742E0230AD072D02840083130008B500D7
:100B9000840A0008B600B10131083507C8003608DC
:100BA000C90048080318C90A232000380319DA2DA0
:100BB000B10ACC2D2E0831020318E02D3108AE0009
:100BC0002E08AF1B0C2EFF3A2F07031C0C2EB00A69
:100BD000B2080319F22D32088400831320308000FC
:100BE000B20AF42D2030DE22AF03E02D36080313C5
:100BF000C90035082320B100B50A0319B60AB00AA6
:100C0000B20803190A2E32088400831331088000C9
:100C1000B20A0C2E3108DE22AE032E0FF62D812EE5
:100C20002B08C9002A0823202A3A031D1E2E023051
:100C3000AD072D028400831300083A2E2B08C9004B
:100C40002A082320D03EAE00AA0A0319AB0A2B08BB
:100C5000C9002A082320B10030303102031C3E2E87
:100C60003A30310203183E2E0A30F1002E08ED22F0
:100C70003107D03EAE00AA0A0319AB0A2B08C900FF
:100C80002A08AA0A0319AB0A2320B100003A031963
:100C9000E02C2A3A0319E92C043A0319102E763A6B
:100CA0000319F22C3B3A0319B42D073A0319F02C1F
:100CB0000B3A0319F42C1C3A0319C12D063A0319F7
:100CC000F62C0D3A0319F22C30303102031C742E2D
:100CD0003A3031020318742E0A30F1002F08ED2249
:100CE0003107D03EAF003E2EB00AB20803197F2E66
:100CF00032088400831331088000B20A812E310843
:100D0000DE222B080313C9002A08AA0A0319AB0A1A
:100D10002320B100B108031DD72CB2080319942E6B
:100D20003208840083138001300808008408031906
:100D30000034720880008403710880008403700806
:100D400080000034F201F11BF2037208F300AB2EB5
:100D5000F201F301B02EF31FB02E7814E127B12E6B
:100D6000F8018E30F6008401F3080319882F031070
:100D7000F30CF20CF10CF00CF60AB42E76087702A4
:100D8000031CCD2E031908000310F20CF10CF00C1B
:100D9000F60A76087702C22E0310F50CF40CF30C59
:100DA000F70A7608770603190800CC2E8030F5067E
:100DB00084015E276D27BE267818E127F81CE82EEF
:100DC000F309F409F509F30A0319F40A0319F50AFA
:100DD0007308F00774080318740FF10775080318F7
:100DE000750FF207F801F21F882FE1277814882F7A
:100DF0008030F5060008F000840A0008F100840A3B
:100E00000008F200D92E84015E276D27F901FA014E
:100E1000FB01F60803190800770803190800760299
:100E2000773EF600780CF8061830F5000310F90D3F
:100E3000FA0DFB0D7208031D252F74087102031DA6
:100E4000232F73087002031C2F2F7308F0027408FD
:100E5000031C740FF102031CF20379140310F00D4C
:100E6000F10DF20DF50B162F7908F0007A08F1005C
:100E70007B08F200882F84015E27F3018230F60799
:100E8000F61B692FF030F607F61B572F1830760245
:100E90000318692FF608031D502F7818E127080062
:100EA000F6030310F00DF10DF20DF30D4A2F0310B0
:100EB000F20CF10CF00CF60F572F4D2FF801710DBD
:100EC000720DF60000380319692FF80DF201F117C1
:100ED0000800F001F101F2010034F810740D750DF5
:100EE000F70000380319792F0318F814F501F417E7
:100EF0000800F701F301F401F50108007608031971
:100F0000692FF113F80C760CF2000318F117962EE6
:100F1000F608031D9C2FF001F101F201962E7203D9
:100F20000319F00A0319F10A0319F20A0310F20C6B
:100F3000F10CF00CF60A882FF208031D8F2F7008B1
:100F4000710403198B2FF11B7E2FF6030310F00D94
:100F5000F10DA32FF601F401F501720873040319D2
:100F600000341F30F6040310F60AF20DF30D031CD3
:100F7000B42FF30CF20C73087102031DC12F720819
:100F80007002031CC92F7208F0027308031C730A55
:100F9000F102F40DF50DF60BF61AB92FF61FD52F49
:100FA000F409F40A0319F503F5097408F200750849
:100FB000F300761F0034F009F00A0319F103F10978
:100FC00000340310FF30F007F009031CF107F109AA
:100FD000031CF207F209031CF307F309080020348D
:100FE0002034203420342034203420342034203461
:100FF0002034203420342034203420342034003471
:02400E0070FF41
:00000001FF
